:020000020000FC
:100000000C94A3160C942A000C942D000C94300030
:100010000C9433000C9434000C9437000C9438008A
:100020000C9439000C943C000C943D000C943E0060
:100030000C943F000C9440000C9441000C9444003C
:100040000C9445000C9446000C9447000C94480016
:100050000C9449000E947B0618950E947B06189517
:100060000E944B09189518950E94E009189518955B
:1000700018950E94470A189518951895189518957F
:1000800018950E94F10A18951895189518951895C5
:1000900018951895600002006200020064000200DA
:1000A000660001009A0001009B000100CE000200E2
:1000B000D00002002F0102003101020033010200D2
:1000C000390102003B0102003D010200670001000E
:1000D000440101004D01020055010200B800010079
:1000E000910001005701020059010100BB0002000C
:1000F0000000772828230852000000000100983AE9
:10010000983A983A983A1400C832684214000100AC
:100110000200DA1FB70F00000000F30F0200B80161
:10012000A8E0B0E0E4E9F0E0C591D5910C2F0D2BEB
:1001300021F0059131960BD0F7CF00916000073781
:1001400021F400916100083209F00FD008951FB723
:10015000F894E199FECFBFBBAEBBE09A2DB32993D3
:1001600011960A95B1F71FBF0895E4E9F0E0A2EFF8
:10017000B0E0C591D5910C2F0D2B71F00591319602
:100180009F01FD01402F159119930A95E1F740FD5C
:100190003196DF01F901EDCF2BD00895A0916200D7
:1001A000B09163000895A0916400B0916500089536
:1001B00000916600017001300895009167000170A0
:1001C000013008951FB71FBFE199FECFF894E19960
:1001D000FACFBFBBAEBBE09A2DB33991231719F00C
:1001E0003DBBE29AE19A11960A9569F71FBF0895FF
:1001F000A8E0B0E0E4E9F0E0C591D5910C2F0D2B1B
:1002000021F005913196DEDFF7CF0895019111912C
:100210000A171B0710F48D0104C0C017D10708F49A
:100220008E01129302930895BEDFED01B7DFEEEC6D
:10023000F0E0ECDFE0EDF0E0E9DFEFE2F1E0E6DF57
:10024000E1E3F1E0E3DFE9E3F1E0E0DFEBE3F1E05C
:10025000DDDF08950C9446010C9447010C946A016B
:100260000C9470010C9497010C94C2010C943F0201
:100270000C94D2030C94D3030C94D9030C94DA039A
:100280000C94DB030C94DC030C941802089500E03A
:1002900010E00E941309E0EBF2E00E940B0900E07D
:1002A00011E00E941309E2ECF2E00E940B090895AC
:1002B00020205365747570202020202020202020CD
:1002C000000020202020202020202020202020206E
:1002D0002020000061E0772704E00E94BF04089519
:1002E00070FD04C06623F9F06A951DC0673071F097
:1002F000FC01A191B1910E941F081127A01BB10B15
:1003000010F4AA27BB27B293A2930DC00091B800A6
:10031000002349F00F3F11F406E001C00A95009355
:10032000B8000E94630B04E00E94BF04089570FDB2
:1003300004C06A30F0F4639521C0673071F0FC01AD
:10034000A191B1910E941F081127A00FB11F10F4B5
:10035000AFEFBFEFB293A29311C00091B800063087
:1003600010F00FEF01C003950093B8000E94630BDB
:1003700005C00CE000938E000E941E0404E00E9461
:10038000BF040895662329F44FDF05E00E94E104CD
:100390004BC0613041F40091660011E001270093E9
:1003A000660026DF41C0623039F40091670011E039
:1003B00001270093670038C0633029F401E07027FB
:1003C0008DE491E031C0643029F401E0702787E5C5
:1003D00091E02AC0653029F401E0702785E591E0BD
:1003E00023C0663049F4009159010395033008F0A9
:1003F00000270093590118C0673019F401E07027F5
:1004000013C0683039F4009191001FEF0127009369
:1004100091000AC0693029F401E070278BEB90E06D
:1004200003C06A3009F400C004E00E94BF040895CC
:100430006A3091F400E010E00E941309EAE5F4E06C
:100440000E940B0900E011E00E941309ECE6F4E0C1
:100450000E940B090E94B50008950420446566615E
:10046000756C742076616C75657300000520686199
:100470007665206265656E2073657420000000E07B
:1004800010E00E941309E8E2F6E002E1069FE00DA9
:10049000F11D0E940B0900E011E00E941309662380
:1004A00019F4EEEEF6E024C0613011F481DE19C0DB
:1004B000623011F482DE15C0663008F450C0663038
:1004C00009F419C0673009F421C0683019F40091AB
:1004D000910007C0693009F478C06A3009F49FC000
:1004E000A2C0002319F4E0E0F7E002C0E2E1F7E087
:1004F0000E940B0998C0EEE6F7E002E11091590165
:10050000019FE00DF11D0E940B098DC005E070FDFB
:1005100008E00E949A0800E20E949A080E949A0845
:100520000E949A080091B800002341F00F3F49F063
:1005300000630E949A08EEE3F7E005C0EAE4F7E002
:1005400002C0E8E5F7E00E940B0970FF6CC000E014
:1005500010E00E94130900E20E949A0864C070FD36
:1005600005C0E4E2F7E00E940B095DC008E00E94CC
:100570009A0800E20E949A08FC01A191B1910E94A0
:10058000AE07A0914701B0914801C0914D01D091B3
:100590004E01633041F0A0914F01B0915001C091E4
:1005A0005501D09156010E945716E6E3F7E06330FB
:1005B00011F0EAE3F7E00E940B0900E010E00E946E
:1005C000130900E20E949A082EC005E070FD08E0C1
:1005D0000E949A0800E20E949A080E949A08A0913C
:1005E000BB00B091BC00CC27DD27E4E6F0E00E9420
:1005F0002F080E94A3070EE20E949A08D4010E94CD
:10060000A707E6E6F7E00E940B0970FF0CC000E0C8
:1006100010E00E94130900E20E949A0804C0E4E27C
:10062000F7E00E940B09089504204578697420536F
:10063000657475703F202020000004204175746FA0
:10064000736176653F20202020200000042045783B
:10065000706F6E656E7469616C3F2020000004202D
:1006600041646A20766F6C74206761696E200000B7
:10067000042041646A207A65726F2063757272206B
:100680000000042041646A2063757272206761690A
:100690006E200000042043757272656E7420696ECE
:1006A00070757420000004204261636B6C69676898
:1006B000742074696D65000004204B6E6F622072B7
:1006C0006576657273653F20000004204C6F7720CB
:1006D00062617474657279202020000004205265E4
:1006E00073657420736574757020202000002020CD
:1006F0005075736820746F2065786974202000003D
:1007000005202020204E6F20202020202020202087
:100710000000052020202059657320202020202063
:100720002020000005202020202020202020202024
:1007300020202020000020562000204120003020D2
:100740007365636F6E6473202000416C7761797309
:10075000206F666620200000416C77617973206FFE
:100760006E20202000002056202020202000052080
:10077000556E69706F6C617220202020202000006F
:1007800005204269706F6C6172202B202020202090
:10079000000005204269706F6C6172202D202020BE
:1007A00020200000089570FF03C004E00E94BF04F1
:1007B000089508950895089508950C94F9030C94EC
:1007C0001D040C941E040C94BE0B0C94FA0B0C9498
:1007D0003B0C0C94630C0C949A0C0C949B0C0C9496
:1007E0009C0C0C947B0C0C949D0C0C949E0C0C9407
:1007F0009F0C0895E2E6F0E0E093BE00F093BF00A6
:10080000E6E4F8E0E093C500F093C600E5E3F4E029
:10081000E093C700F093C80000270093680008EE3B
:1008200013E00093C9001093CA000E94D300A09364
:10083000CB00B093CC0085E008950895DBDF0E94E3
:10084000B20B61E00895202050574D206C6F772047
:100850006C696D6974200000202050574D20686934
:100860006768206C696D6974000010916800003041
:1008700029F4112309F448C01A9504C0113009F471
:100880004DC01395109368001030F1F4E2E6F0E0EB
:10089000E093BE00F093BF00E6E4F8E0E093C5000B
:1008A000F093C600A8EEB3E0A093C900B093CA00CD
:1008B0000E94D300A093CB00B093CC0085E061E010
:1008C000003009F465E02AC0113041F5E4E6F0E0BB
:1008D000E093BE00F093BF00E8E5F8E0E093C500C8
:1008E000F093C6000E94CE00A093C900B093CA0046
:1008F000A8EEBDEFA093CB00B093CC0085E061E003
:10090000003009F465E00AC00E94CA0A0BE00093B7
:100910008E006AE0772704E00E94BF04089509E68C
:1009200010E00093890010938A0000938B001093CD
:100930008C00002700938D0008951F932F93EF9351
:10094000FF932FB7F89410918D00103290F4139507
:1009500010938D00E0918900F0918A000193E938AD
:1009600021F4F03011F4E9E6F0E0E0938900F0932F
:100970008A002FBFFF91EF912F911F9108951F9330
:100980002F933F93EF93FF933FB7F89410918D000F
:10099000112379F0E0918B00F0918C0021910217E6
:1009A00049F0E93821F4F03011F4E9E6F0E01A9565
:1009B000A9F7C3DF3FBFFF91EF913F912F911F91A7
:1009C00008951F932F93EF93FF932FB7F8941091EF
:1009D0008D00103290F4139510938D00E0918B00F0
:1009E000F0918C00E93621F4F03011F4E9E8F0E000
:1009F0000293E0938B00F0938C002FBFFF91EF9157
:100A00002F911F9108951F93EF93FF93E8941FB7C1
:100A1000F89400918D00002399F00A9500938D00C1
:100A2000E0918B00F0918C000191E93821F4F030D5
:100A300011F4E9E6F0E0E0938B00F0938C00106491
:100A40001FBFFF91EF911F910895380D820DCC0DBE
:100A50001E0EB20E271173120A150C14C3142A01AC
:100A6000DD030E948F040AE00093900000270093AA
:100A70008E0001E000938F000CE0EAE4FAE0C591FB
:100A8000D5912096EF93FF930F93FE0109950F9157
:100A9000FF91EF910A9599F708950E9403050EF0D2
:100AA000089510918E00013009F422C0023009F43B
:100AB00032C0033009F442C0043009F44DC005309F
:100AC00009F471C0063009F47CC0073009F49CC0F9
:100AD000083009F4A7C0093009F4AFC00A3009F49E
:100AE000B1C00B3009F4C2C00C3009F4CBC008957A
:100AF0000E94630B10918E00112311F003E0C7C018
:100B000010918F001A9509F4139510938F0004E04B
:100B10000E94BF0408950E94630B10918E00112360
:100B200011F004E0B4C010918F001B3008F413954D
:100B300010938F0004E00E94BF0408950E94630B8D
:100B400010918E00112311F005E0A1C010918F00CB
:100B500010938E0002E09BC0112339F006E097D07D
:100B60000E94A90BF9F4AAD01DC010918F0001E0DA
:100B70008ED00E94A90B11F4A1D00BC020918F0040
:100B8000213039F000E010E00E94130902E00E94D9
:100B90009A082B3039F000E011E00E94130903E0BD
:100BA0000E949A0808950E94CA0A112710938E0085
:100BB0000E94D80011F40E94F80004E00E94BF04D3
:100BC00008950FB7F894A0919E00B0919F000FBFB9
:100BD000A093D200B093D3000E94800EA091D200C7
:100BE000B091D3000E94FA0E10918E00112311F0E3
:100BF00007E04DC000918F00033011F0043019F46C
:100C000004E00E94BF0408950E94CE0A0E944B0B8C
:100C10000E94770B60D010918E00112311F008E034
:100C200036C008950E943F150E94930B10918E00CC
:100C3000112311F009E02BC00895112311F00AE0EF
:100C400026C008950E94A7110E94F31210918E00F1
:100C5000112311F00BE01BC000918F00063011F042
:100C6000073019F404E00E94BF040895112311F025
:100C70000CE00DC000918F00093019F404E00E94CF
:100C8000BF040895112311F00DE001C00895112350
:100C9000A1F01A951C3088F42227110F221FEAE4D4
:100CA000FAE0E10FF21FC591D591E02FFF27EE0F7B
:100CB000FF1FEC0FFD1F09950895089500E010E057
:100CC0000E94130902E410919000163008F400E22B
:100CD0000E949A080895009190000A9509F40AE08C
:100CE000009390000A3011F0053021F40E94A90B06
:100CF00009F4E4DF08950F930FB70F931F932F9319
:100D000000B3102F1695102712FD24C010919300E8
:100D1000102712FF2BC01091930000939300209195
:100D20009600222309F422C02227209396000695DC
:100D30000695102700919100102701E010FD02E0B8
:100D40000E949D04009195000093920004E100939D
:100D500095000CC021E020939600109193001C7F19
:100D6000069506950370012B009393002F911F9118
:100D70000F910FBF0F91089500B300781091940068
:100D800016951F77012B00939400007F003121F40A
:100D900003E00E949D0411C0002361F400919700BC
:100DA000002359F00A950093970039F40CE00E9453
:100DB0009D0403C000E500939700009195000A95FB
:100DC00012F000939500089501B3037701BB02B3BD
:100DD000037702BB05B7007F056005BF0BB7006C4A
:100DE0000BBF00B3009393000FEF00939400002714
:100DF00000939200009395000093960000E5009305
:100E0000970008950F93000000000000000000000C
:100E1000000000000A95B9F70F9108950F930AEFAB
:100E2000F1DFF0DFEFDFEEDF1197D1F70F910895DB
:100E30000027AC17BD0720F00395AC1BBD0BF9CF05
:100E400008950F93C0E1D7E2F3DF00630E949A0890
:100E50000EE20E949A08C8EED3E0EADF00630E9427
:100E60009A08C4E6D0E0E4DF00630E949A08CAE072
:100E7000D0E0DEDF00630E949A080A2F00630E9420
:100E80009A0800E20E949A080DE60E949A0803E779
:100E90000E949A080F910895ED010E94CE00CA1B8E
:100EA000DB0BFD01A7E3BB270E944D080E94D30086
:100EB000AE1BBF0BFD01D801E9010E942F08A7332B
:100EC00008F0A6E3089588249924AA24BB24CC24FE
:100ED000DD24EE24FF24089533952695A8F420E11F
:100EE000992049F40F9302E0882009F403E00E945E
:100EF0009A080F9108C00F93042F0E942A090E949C
:100F00009A080F914395DFDF0895822A922AA22A38
:100F1000B22AC22AD22AE22A089520E1332744E0E5
:100F20005527D1DF552311F4E22A01C0822A301758
:100F300011F45FEFEADF311711F45527E6DFCCDF5C
:100F4000373381F708950F936894BB2721C00F931F
:100F5000E894BB2729C00F93BB2730C00F93689438
:100F6000C0E1D7E265DF00632EF4E894003311F4AA
:100F7000689400E20E949A08C8EED3E059DF00634B
:100F80002EF4E894003311F4689400E20E949A0869
:100F9000C4E6D0E04DDF00632EF4E894003311F492
:100FA000689400E20E949A08CAE0D0E041DF006342
:100FB0001EF4003309F400E20E949A080A2F00632D
:100FC0000E949A080F91089501000A006400E80346
:100FD00010270F93EF93FF93E8ECFFE0000FE00F73
:100FE0000027F01FA591B491FF91EF910F91089503
:100FF00001010101010101010101020203030404D5
:101000000505EF93FF930E94DD0061F400919200CB
:10101000013108F000E1E0EFFFE0E00F0027F01FF2
:10102000049101C001E0FF91EF91089501010101D8
:101030000101010101010A0A0A0A0A0A6464EF9324
:10104000FF9300919200013108F000E1ECE2F0E141
:10105000E00F0027F01F0491FF91EF910895CC2439
:1010600088249924AA24BB1801E2AA1FBB1FCC1F05
:10107000DD1F0A9509F40895881C991CAA1CBB1C45
:101080008E1A9F0AAC08BC0830F48E0E9F1EAC1C52
:10109000BC1C8894EACF0894E8CF4427BD9F9001F8
:1010A000AC9F8001BC9F100D211D341FDA9F100DD5
:1010B000211D341F0895007FC39A18B31F70102B91
:1010C00018BBC39808951F930F93F5DF01E00E94AA
:1010D00002070F910F930295EEDF0BE20E940207C9
:1010E0000F911F910895C39A0000000000000000B6
:1010F000000006B3C398007F08951F9318B3106FC4
:1011000018BB17B31F7017BBEEDF102F00000000D5
:10111000000000000000E7DF0295102B0BE20E94A8
:101120000207012F17B3106F17BB1F910895C198C5
:10113000C298C9CFC19AC298C6CFC198C29ADDCF12
:10114000C19AC29ADACF0F931F9307B30E6F07BBF2
:10115000AFE0BB270E940E0700E3ADDFA5E0BB2791
:101160000E940E0700E3A7DF04E60E94020700E3E7
:10117000A2DF08E20E94020700E29DDF08E20E946F
:10118000020708E2D4DF06E0D2DF0CE0D0DF01E0A6
:10119000CEDFA2E0BB270E940E0705D000E8C7DF24
:1011A0001F910F910895EEEBF1E102C0E6EFF1E13E
:1011B00000E4BDDF0591BEDF07FFFCCF0895040406
:1011C0001F0404001F000001020204140800040EA2
:1011D00015040404040004040404150E04000004AF
:1011E000021F020400000004081F080400001F1F63
:1011F0001F1F1F1F1F8004041F0404001F00000185
:101200000202041408001F0000000000000000009B
:10121000000000001F800F930591002311F08ADF6A
:10122000FBCF0F9108950F931F930F7011701295BC
:10123000110F110F010F00687ADF1F910F910895B0
:101240000F930FE074DF0F9108950F930CE06FDFA1
:101250000F9108951F930F930F936FDF102F0F912E
:10126000000F000F000F006462DF082D63DF092DFF
:1012700061DF0A2D5FDF0B2D5DDF0C2D5BDF0D2D98
:1012800059DF0E2D57DF002755DF012F00684FDF94
:101290000F911F9108950F930FB70F931F93009114
:1012A00099000395043009F401E00093990001705E
:1012B000005A03BD0E94BC060E94210A00919800BA
:1012C0000A950093980051F40AE0009398000E9458
:1012D000310A0E94BF1307E00E949D041F910F91E5
:1012E0000FBF0F9108950AE000939800002702BDF8
:1012F00004BD009399000FE005BD00E603BD09B7EA
:1013000000680F7B09BF089506E000939C000093DE
:101310009D0008951F9310919A00011307C010912A
:101320009C0010939A0000939C0004C000939A00C4
:1013300010939C001F9108951F9310919B0001131F
:1013400007C010919D0010939B0000939D0004C066
:1013500000939B0010939D001F910895003029F485
:101360000091CE001091CF000895013029F4009132
:10137000D0001091D1000895023029F400919E0010
:1013800010919F000895033029F40091D40010912A
:10139000D5000895043029F400912D0110912E01FB
:1013A0000895053029F4009137011091380108950E
:1013B000063019F4002711270895002711270895F2
:1013C0000F930FB70F931F93AF93BF930EB510E416
:1013D00001270EBD06FD07C006B517B50093A00096
:1013E0001093A10027C006B517B5A091A000B09139
:1013F000A1000A1B1B0B0E94CE000A171B07A8F0B6
:101400000E94D300A017B10798F000939E0010939C
:101410009F0006E00E949D040AE00093A300009153
:10142000A40003950093A40005C00E94470F02C0CA
:101430000E94620FBF91AF911F910F910FBF0F914B
:1014400008951091A3001A9549F41AE0002700931B
:101450009E0000939F0006E00E949D041093A3004D
:1014600008950091A4001091A500101750F0039565
:10147000011748F4AF93BF930E947D0FBF91AF91C6
:1014800000270093A50000270093A40008950F9360
:101490000FB70F931F931091A200103031F011304D
:1014A00039F11230C1F1112737C0139500270BBD58
:1014B0000ABD09BD08BD1F932F9320EA00919A0031
:1014C0000E94AE090093A6001093A700012B09F01B
:1014D000206400919B000E94AE090093A800109325
:1014E000A900012B09F020612FBD2F911F9114C07D
:1014F00013950091A7000BBD0091A6000ABD0091B5
:10150000A90009BD0091A80008BD00EA0FBD0AE0CE
:101510000E94E10401C011271093A2001F910F91B6
:101520000FBF0F91089500270093A20000939E0023
:1015300000939F000093A4000093A5000AE000938D
:10154000A30000EA0FBD0C600FBD01EC0EBD09B792
:101550000462077E09BF01B3006301BB969A089538
:1015600000270093AA0008950F930093AB001093F7
:10157000AC000E941309022F0E949A083093AD001C
:101580000091AA0001600093AA000AE00093AE0057
:101590000F91089500270093AA0008950091AA00D2
:1015A00000FF1EC00091AE000A950093AE00C1F48A
:1015B00004E00093AE000091AB001091AC000E94DB
:1015C00013090E94A0082091AD000093AD00009186
:1015D000AB001091AC000E941309022F0E949A08E0
:1015E00008950F930FB70F931F932F933F9300917D
:1015F000B70003950093B7000130F1F10A3038F0DD
:1016000099F00D30C8F10531A0F001F135C004B1F9
:1016100015B12091B3003091B400200F311F2093F9
:10162000B3003093B40028C007B1017E016007B950
:1016300023C004B115B12091B5003091B600200F40
:10164000311F2093B5003093B60016C006B10F7954
:1016500006B90091B3001091B4000093AF0010934D
:10166000B0000091B5001091B6000093B100109346
:10167000B20008E00E949D043F912F911F910F91AD
:101680000FBF0F91089500E007B90FE806B900B742
:101690000F7100BF08950AB30C7F0ABB0BB30C7F18
:1016A0000BBB00270093B3000093B4000093B50078
:1016B0000093B6000093B70007B1007E07B906B1EA
:1016C000006606B908950091B800002371F00F3F3D
:1016D00019F40FEF1FEF03C014E6019F8001009380
:1016E000B9001093BA00AE9A01C0AE980895A091C7
:1016F000B900B091BA000A2F0B230F3F39F01197B0
:10170000A093B900B093BA0009F4AE980895A69AD0
:10171000AE9800270093B9000093BA0008950027FF
:101720000093BD000895A0914701B0914801C09178
:101730004D01D0914E010E944D08A091BB00B09187
:10174000BC0000272A173B0708F401E00093BD0006
:1017500008950091BD0001700130089500270093A5
:10176000CD0008956627772701E00093CD0004E0BF
:101770000E94BF0409E00E94BF04089570FD12C0DA
:10178000662389F16A9529F080FD2DC0653059F5F1
:10179000662782FF28C0E091C700F091C80000E0F2
:1017A000099521C005E0061B0E94E907E091BE00F3
:1017B000F091BF00C191D1910E940108CA1BDB0BBF
:1017C00018F00A95D9F702C0DD27CC27DE010E9468
:1017D0000A0D21F0A091C900B091CA000FB7F8948A
:1017E000B293A2930FBF04E00E94BF0409E00E94DD
:1017F000BF04089570FD17C0673060F4062F03958D
:10180000013011F480FF06E0063011F481FF02C0C0
:10181000602F2AC082FF28C0E091C700F091C80065
:1018200001E0099521C005E0061B0E94E907E0914F
:10183000BE00F091BF00C191D1910E940108CA0F72
:10184000DB1F18F00A95D9F702C0DFEFCFEFDE01FA
:101850000E940A0D21F0A091CB00B091CC000FB7EF
:10186000F894B293A2930FBF04E00E94BF0409E072
:101870000E94BF040895662339F400270093CD0029
:1018800005E00E94E1041EC0663060F401E07027AC
:101890007B7F0E94D30804E00E94BF0409E00E94FD
:1018A000BF0410C00091C400663019F40E948A0978
:1018B00002C00E949C09726004E00E94BF0409E01B
:1018C0000E94BF0408950E94CA0A4CD024E035E06B
:1018D00070FF02C020E238E000E010E00E9413092F
:1018E000022F0E949A0800E011E00E941309032FC2
:1018F0000E949A08089572FD1BC0062F613038F0CF
:101900000395623020F00395663008F00A5F11E01D
:101910000E9413090F930E94A008202F0F9136E018
:1019200070FD04C071FD02C0322F26E00E94B40A8F
:101930007D7F0895089508950895089508957B7F03
:101940000E94D30883FF0DC0662359F0663048F427
:1019500075600E94D60804E00E94BF0409E00E945E
:10196000BF0408950E94250900E010E00E941309B9
:10197000E091C500F091C6000E940B0900E011E063
:101980000E941309ECE0FAE10E940B09E091BE000D
:10199000F091BF00A191B1910091CD000023D9F049
:1019A00072FF19C0E091C000F091C100A191B19106
:1019B0000E944C07AF93E091C200F091C300A19147
:1019C000B1910E944C071A2F0F910E948D0700E2DF
:1019D0000E949A0806C00E942107E0E1FAE10E94F5
:1019E0000B0901E010919A002091C400121300E24B
:1019F00081FF00E20E949A0801E010919B001213FF
:101A000000E281FF00E20E949A0808952020000071
:101A100020202000CF93DF93C091C900D091CA004D
:101A2000AC17BD0748F0C091CB00D091CC00CA17CD
:101A3000DB0710F0189401C09894DF91CF910895BE
:101A40000E94CE00A093C900B093CA000E94D300A8
:101A5000A093CB00B093CC00089500270093C90059
:101A60000093CA000FEF0093CB000093CC000895C1
:101A70000C94540D0C94710D0C94750D0C94BE0BBC
:101A80000C94FA0B0C943B0C0C94630C0C949A0C75
:101A90000C949B0C0C949C0C0C947B0C0C949D0C47
:101AA0000C949E0C0C949F0C0895EEECF0E0E093E7
:101AB000BE00F093BF00E093C000F093C100E0933C
:101AC000C200F093C300E2EFFAE1E093C500F093A7
:101AD000C60000E00093C4000E94200D77278BE031
:101AE0000895E3DF0E94B20C0895DFDF0E94B20B7D
:101AF000089520204F7574707574203120202020A7
:101B0000414200000C949E0D0C94BB0D0C94BF0D33
:101B10000C94BE0B0C94FA0B0C943B0C0C94630CC1
:101B20000C949A0C0C949B0C0C949C0C0C947B0CB9
:101B30000C949D0C0C949E0C0C949F0C0895E0ED5D
:101B4000F0E0E093BE00F093BF00E093C000F0939C
:101B5000C100E093C200F093C300E6E8FBE1E0932C
:101B6000C500F093C60001E00093C4000E94200D60
:101B700077278BE00895E3DF0E94B20C0895DFDF42
:101B80000E94B20B089520204F7574707574203236
:101B900020202020414200000C94E80D0C94020EFD
:101BA0000C94060E0C94BE0B0C94FA0B0C943B0C8C
:101BB0000C94630C0C940A0E0C949B0C0C949C0CCF
:101BC0000C947B0C0C949D0C0C949E0C0C949F0C10
:101BD00000270093D2000093D3000895E2EDF0E0D7
:101BE000E093BE00F093BF00EAE2FCE1E093C500A1
:101BF000F093C60002E00093C4000E94200D7727F6
:101C000082E00895EBDF0E94B20C0895E7DF0E94A6
:101C1000B20B089502E011E00E941309A091D200D6
:101C2000B091D3000E94210708952020496E70755D
:101C30007420202020202020414200000C943A0EE5
:101C40000C94640E0C94680E0C94BE0B0C94FA0B5E
:101C50000C943B0C0C94630C0C946C0E0C949B0C2D
:101C60000C949C0C0C947B0C0C949D0C0C949E0C72
:101C70000C949F0C00270093D4000093D500009390
:101C8000D6000093D7000093D800E9EDF0E0E09390
:101C90001901F0931A0110E401931A95E9F70895D8
:101CA000E4EDF0E0E093BE00F093BF00EEEEFCE167
:101CB000E093C500F093C60003E00093C4000E94C7
:101CC000200D772782E00895EBDF0E94B20C089583
:101CD000E7DF0E94B20B089502E011E00E941309B1
:101CE000A091D400B091D5000E9421070895202032
:101CF000496E707574206176672E20204142000085
:101D00000091D6001091D7002091D800E0911901E0
:101D1000F0911A01C191D19133270C1B1D0B230B9C
:101D20000A0F1B1F231FB293A2930093D600109398
:101D3000D7002093D80035E02695179507953A955A
:101D4000D9F70093D4001093D5003296C9E1D1E0C1
:101D5000EC17FD0710F0E9EDF0E0E0931901F093C6
:101D60001A0108950C94CE0E0C94980F0C94BB0F8E
:101D70000C94C00F0C94C70F0C94CE0F0C94D90F79
:101D80000C941D110C9421110C9422110C9423110C
:101D90000C9424110C9425110C94261101D0089553
:101DA0000FEF00931B0100931C01002700931D01FE
:101DB00000931E011FB7F89400931F0100932001A8
:101DC0000093210100932201009323010093240139
:101DD0000093250100932601009327010093280119
:101DE0000093290100932A0100932B0100932C01F9
:101DF0001FBF08950A2F0B2BB9F0C0911B01D09182
:101E00001C01AC17BD0720F4A0931B01B0931C016B
:101E1000C0911D01D0911E01CA17DB0720F4A093C9
:101E20001D01B0931E0101D008950FB7F894A09141
:101E30002301B09124011196A0932301B0932401B2
:101E400020F5A0E0B0E8A0932301B0932401A09175
:101E50002101B0912201B695A795A0932101B093DD
:101E60002201A0912901B0912A01B695A795A093CE
:101E70002901B0932A01A0912B01B0912C01B695B4
:101E8000A795A0932B01B0932C010FBF08950FB716
:101E90000F93F894A0912501B0912601119620F09E
:101EA000A0932501B0932601A0912901B0912A01A8
:101EB000119620F0A0932901B0932A01B6DF0F916B
:101EC0000FBF08950FB70F93F894A0912701B09119
:101ED0002801119620F0A0932701B0932801A0912A
:101EE0002B01B0912C01119620F0A0932B01B093FF
:101EF0002C019BDF0F910FBF08950FB70F93F8943C
:101F0000A0911F01B0912001119620F0A0931F0114
:101F1000B0932001A0912101B0912201119620F0EF
:101F2000A0932101B093220180DF0F910FBF08958C
:101F300000E010E00E941309E2E5FFE10E940B09B6
:101F400000E011E00E941309E4E6FFE10E940B09A2
:101F500008952020496E7075742053746174202098
:101F600020200000202020202020202020202020B1
:101F700020202020000061E004E00E94BF040895BA
:101F8000662309F06A9504E00E94BF040895663054
:101F900008F4639504E00E94BF040895662321F4C9
:101FA00005E00E94E10404C0FBDE04E00E94BF04DF
:101FB000089500E010E00E941309E8E4F1E202E174
:101FC000069FE00DF11D0E940B0900E011E00E9448
:101FD0001309662329F4E6ECF1E20E940B09B3C071
:101FE0006130B9F400911B0110911C0101230F3FD6
:101FF00009F4A5C0E8EDF1E20E940B09A0911B01D4
:10200000B0911C010E942107ECEDF1E20E940B0946
:102010009AC06230B9F400911B0110911C01012398
:102020000F3F09F48CC0E8EDF1E20E940B09A0918A
:102030001D01B0911E010E942107ECEDF1E20E940A
:102040000B0981C0633001F500911B0110911C0147
:1020500001230F3F09F473C0E8EDF1E20E940B0980
:10206000A0911D01B0911E01C0911B01D0911C01D6
:10207000AC1BBD0B10F4AA27BB270E942107ECED77
:10208000F1E20E940B095FC06430E9F4E8EDF1E28F
:102090000E940B090FB7F894A0911F01B091200185
:1020A0000FBF0E94AE0700E20E949A080FB7F89493
:1020B000A0912101B0912201E0912301F09124012E
:1020C0000FBF98D040C06530E9F4E8EDF1E20E941E
:1020D0000B090FB7F894A0912501B09126010FBF0D
:1020E0000E94AE0700E20E949A080FB7F894A091F0
:1020F0002901B0912A01E0912301F09124010FBF41
:1021000079D021C0E8EDF1E20E940B090FB7F894F5
:10211000A0912701B09128010FBF0E94AE0700E2F5
:102120000E949A080FB7F894A0912B01B0912C014E
:10213000E0912301F09124010FBF5CD004C0E2EED6
:10214000F1E20E940B090895042050757368207411
:102150006F2065786974202000000420496E707536
:1021600074206D696E696D756D2000000420496EE4
:10217000707574206D6178696D756D2000000420A4
:10218000496E707574206A6974746572202000004D
:102190000420496E7075742064726F706F7574736B
:1021A00000000420496E70757420746F6F206C6F8E
:1021B000772000002020496E70757420746F6F20A6
:1021C000686967680000202020496E70757420538C
:1021D00074617420202000000520000020202020B1
:1021E000200005204E6F2076616C696420696E7056
:1021F000757400000E2F0F2B29F4AA27BB27882403
:1022000099240CC0C0E1D7E20E944D08D801E90131
:102210000E942F08E4E6F0E00E942F080E94A30726
:102220000EE20E949A08D4010E94A70700E20E94D1
:102230009A0805E20E949A08089504E00E94BF04EB
:1022400008950895089508950895089508950C94A3
:1022500043110C946C110C9470110C94BE0B0C94E3
:10226000FA0B0C943B0C0C94630C0C949A0C0C948D
:102270009B0C0C949C0C0C947B0C0C9474110C9483
:102280009E0C0C949F0C00912F0100932D01009146
:10229000300100932E0100E0009336010895EDE235
:1022A000F1E0E093BE00F093BF00E6E0F3E2E093DC
:1022B000C500F093C60004E00093C400ECEDF1E12A
:1022C000E093C700F093C8000027009335010E94F7
:1022D000200D772786E00895E2DF0E94B20C089572
:1022E000DEDF0E94B20B089500913501002351F406
:1022F00002E011E00E941309A0912D01B0912E017E
:102300000E942107089520205377656570203120B1
:10231000202020204142000020204C6F77206C6953
:102320006D69742020202020000020204869676803
:10233000206C696D697420202020000020205374D7
:1023400065702F7370656564202020200000E09187
:102350002D01F0912E01A0913301B0913401009133
:102360003601003089F4C0913101D0913201EA0F79
:10237000FB1F10F4EFEFFFEFEC17FD0720F0FE015D
:1023800001E00093360110C0C0912F01D0913001BF
:10239000EA1BFB0B10F4EE27FF27CE17DF0720F018
:1023A000FE0100E0009336010FB7F894E0932D0191
:1023B000F0932E010FBF089510913501003029F4DC
:1023C000112309F48FC01A9504C0133009F48AC090
:1023D0001395109335011030A9F4EDE2F1E0E0938C
:1023E000BE00F093BF00E6E0F3E2E093C500F09397
:1023F000C6000E94200D8260867F60E0003009F4F4
:1024000067E070C0113059F5EFE2F1E0E093BE00F3
:10241000F093BF00E093C000F093C100E1E3F1E06E
:10242000E093C200F093C300E8E1F3E2E093C5005B
:10243000F093C6000E94CE00A093C900B093CA00DA
:10244000A0913101B0913201A093CB00B093CC00A8
:1024500089608D7F61E0003009F465E043C012308F
:1024600059F5EFE2F1E0E093C000F093C100E1E341
:10247000F1E0E093BE00F093BF00E093C200F09360
:10248000C300EAE2F3E2E093C500F093C600A09136
:102490002F01B0913001A093C900B093CA000E94EF
:1024A000D300A093CB00B093CC0089608D7F61E016
:1024B000003009F465E016C01330A1F4E3E3F1E065
:1024C000E093BE00F093BF00ECE3F3E2E093C500BD
:1024D000F093C6000E942D0D8160857F61E0003081
:1024E00009F465E008950C948F120C94B8120C94C2
:1024F000BC120C94BE0B0C94FA0B0C943B0C0C9479
:10250000630C0C949A0C0C949B0C0C949C0C0C94E7
:102510007B0C0C94C0120C949E0C0C949F0C00919C
:1025200039010093370100913A010093380100E02E
:10253000009340010895E7E3F1E0E093BE00F093DB
:10254000BF00EEE9F5E2E093C500F093C60005E0B8
:102550000093C400E8E2F3E1E093C700F093C80001
:10256000002700933F010E94200D772786E0089501
:10257000E2DF0E94B20C0895DEDF0E94B20B0895E4
:1025800000913F01002351F402E011E00E94130981
:10259000A0913701B09138010E94210708952020B1
:1025A00053776565702032202020202041420000B2
:1025B00020204C6F77206C696D69742020202020CA
:1025C0000000202048696768206C696D69742020CC
:1025D000202000002020537465702F73706565649F
:1025E000202020200000E0913701F0913801A091D7
:1025F0003D01B0913E0100914001003089F4C0914D
:102600003B01D0913C01EA0FFB1F10F4EFEFFFEF0D
:10261000EC17FD0720F0FE0101E00093400110C01F
:10262000C0913901D0913A01EA1BFB0B10F4EE275F
:10263000FF27CE17DF0720F0FE0100E000934001E6
:102640000FB7F894E0933701F09338010FBF089566
:1026500010913F01003029F4112309F48FC01A951D
:1026600004C0133009F48AC0139510933F01103051
:10267000A9F4E7E3F1E0E093BE00F093BF00EEE9D8
:10268000F5E2E093C500F093C6000E94200D826041
:10269000867F60E0003009F467E070C0113059F5C2
:1026A000E9E3F1E0E093BE00F093BF00E093C000E7
:1026B000F093C100EBE3F1E0E093C200F093C300BC
:1026C000E0EBF5E2E093C500F093C6000E94CE0077
:1026D000A093C900B093CA00A0913B01B0913C0106
:1026E000A093CB00B093CC0089608D7F61E0003077
:1026F00009F465E043C0123059F5E9E3F1E0E093F5
:10270000C000F093C100EBE3F1E0E093BE00F09372
:10271000BF00E093C200F093C300E2ECF5E2E09367
:10272000C500F093C600A0913901B0913A01A09381
:10273000C900B093CA000E94D300A093CB00B0930D
:10274000CC0089608D7F61E0003009F465E016C03F
:102750001330A1F4EDE3F1E0E093BE00F093BF008D
:10276000E4EDF5E2E093C500F093C6000E942D0D64
:102770008160857F61E0003009F465E008952F9362
:1027800022B708B700FF19C001E008BF009142015D
:10279000013041F001E000934201002702BF0093A5
:1027A000430125C00FEF00934101002702BF0093B2
:1027B00043010BE00E949D041AC000914301039560
:1027C0000093430110914201011788F0243130F445
:1027D000013021F40AE00093420109C02093410135
:1027E000002702BF009343010BE00E949D042F913C
:1027F0000895B898C09A00270093410100934301BF
:1028000002BF0AE00093420107E003BF09B70C7F53
:1028100009BF01E008BF08950C94F9130C94281423
:102820000C942A140C9431140C9440140C944F14EE
:102830000C9453140C945E140C945F140C94601458
:102840000C9461140C946E140C946F140C94751405
:102850004DD0089504E00E94BF0409E00E94BF0427
:102860000895009144010A95023008F402E00093B3
:10287000440104E00E94BF0409E00E94BF040895DF
:10288000009144010395053008F004E000934401F1
:1028900004E00E94BF0409E00E94BF04089505E01F
:1028A0000E94E10408950E94CA0A20D000E011E0CD
:1028B0000E94130908E00E949A0808950895089557
:1028C000089509E010E00E9413090F930E94A008E8
:1028D000202F0F9136E00E94B40A0895089502E077
:1028E00011E00E94130931D00895089500E010E02E
:1028F0000E941309EAE2F9E20E940B0900914401E7
:1029000000630E949A08E4E3F9E20E940B0900E0E8
:1029100011E00E941309ECE3F9E20E940B0915D0C3
:10292000E0E4F9E20E940B090895202054616368F5
:102930006F20200020626C61646500002020000090
:102940002072706D202020202000009141012091F4
:102950004401233028F011F01FE003C014E101C04E
:102960001EE1019FD00100914201013049F4CAE00B
:10297000D0E00E944D08D801232B11F0AFEFBFEF3C
:102980000E94AE0708950C94DF140C94F9140C9473
:10299000FD140C94BE0B0C94FA0B0C943B0C0C9491
:1029A000630C0C949A0C0C949B0C0C949C0C0C9443
:1029B0007B0C0C949D0C0C949E0C0C949F0C00278B
:1029C00000934501009346010895E5E4F1E0E093AA
:1029D000BE00F093BF00E2E0FAE2E093C500F0939E
:1029E000C60006E00093C4000E94200D772782E015
:1029F0000895EBDF0E94B20C0895E7DF0E94B20B4E
:102A00000895202044697361626C65206F7574209D
:102A1000414200000C9426150C948F150C94B215AD
:102A20000C94B8150C94BF150C94C6150C94D115C4
:102A30000C9484160C9485160C9486160C948D16A2
:102A40000C948E160C948F160C94901601D0089549
:102A50000FEF0093490100934A010FEF1FE7009326
:102A6000510110935201002700934B0100934C0138
:102A700000E010E8009353011093540108954FB7FC
:102A8000F8940091AF001091B000A091B100B09106
:102A9000B2004FBF00934701109348014091590184
:102AA000442359F0C0915701D0915801AC1BBD0B84
:102AB000423019F4A095B0951196A0934F01B093B0
:102AC00050019D01A0914901B0914A010A171B07CD
:102AD00020F40093490110934A01A0914B01B09159
:102AE0004C01A017B10720F400934B0110934C0147
:102AF000A0915101B09152012A173B0724F4209371
:102B0000510130935201A0915301B0915401A21789
:102B1000B30724F42093530130935401089500E047
:102B200010E00E941309E0E4FBE20E940B0900E0C0
:102B300011E00E941309E2E5FBE20E940B090895EF
:102B40002020566F6C7461676520616E64202020C0
:102B500000002020202063757272656E7420202092
:102B600020200000662775E004E00E94BF0408955D
:102B7000662309F06A9504E00E94BF04089562305C
:102B800008F4639504E00E94BF040895662321F4CD
:102B900005E00E94E10404C05BDF04E00E94BF0482
:102BA000089500E010E00E941309662329F5E0E98A
:102BB000FCE20E940B09A0914701B0914801C0912D
:102BC0004D01D0914E0173D006E50E949A0800E0B5
:102BD00011E00E941309EAE9FCE20E940B09A091AE
:102BE0004F01B0915001C0915501D09156015FD075
:102BF00001E40E949A084BC0613029F5E0E9FCE24B
:102C00000E940B09A0914B01B0914C01C0914D0164
:102C1000D0914E014CD006E50E949A0800E011E0E8
:102C20000E941309E4EAFCE20E940B09A091490109
:102C3000B0914A01C0914D01D0914E0138D006E5C6
:102C40000E949A0824C0EAE9FCE20E940B09A091C4
:102C50005301B0915401C0915501D091560127D034
:102C600001E40E949A0800E011E00E941309E4EADE
:102C7000FCE20E940B09A0915101B0915201C09158
:102C80005501D091560113D001E40E949A0808958D
:102C90000420566F6C746167650020204375727262
:102CA000656E740005206D61782F6D696E00EE27EA
:102CB000BB2322F4EFEFA095B09511960E944D082A
:102CC000D9015E2FCC27DD27E4E6F0E00E942F0833
:102CD00055238AF4AA3048F400E20E949A080DE2D3
:102CE0000E949A080E94AB0708C00DE20E949A0851
:102CF0000E94A70702C00E94A3070EE20E949A0842
:102D0000D4010E94A7070895089508957A9521F4A3
:102D100075E004E00E94BF040895089508950895A1
:102D2000089520536572766F205465737465722020
:102D300032200000202056657273696F6E20312E9C
:102D40003030202000000FE50DBF04E00EBF00E88A
:102D500008B900270ABB07BB04BB01BB1CEF1BBBA8
:102D600008BB13E815BB02BB0E9490000E9431050E
:102D70000E94E4060E94A3080E94B00A0E94730900
:102D80000E9484090E94930A0E94430B0E94AE0B8A
:102D90000E94870B0E948F0B78940E94630B00E0C7
:102DA00010E00E941309E2E2FDE20E940B0900E03C
:102DB00011E00E941309E4E3FDE20E940B090E9466
:102DC0000305EEF338E20E940305EEF7013041F00F
:102DD000023031F0033021F00730A9F73A9599F726
:0C2DE00004E00E949D040E944D05FDCF00
:00000001FF
